:030000000219FDE5
:03000B000200A848
:03002B0002015A75
:03005B000202EEB0
:030073000202DBAB
:1000800002030406080C10182030406080040608A3
:100090000C10182030406080A0C00003070F1F051F
:1000A000050D050305030302C2AFC0D0C0E0206206
:1000B00014E5256009E473E525F4F58AD262D0E001
:1000C000D0D0D2AF3285268AC262E526F4602F30C6
:1000D000682520720DD0E0D0D0C2B1C287C281D2D3
:1000E000AF32C2B1C287C281206F0C206609740A88
:1000F000D5E0FDE57B4280D0E0D0D0D2AF32758A2A
:1001000000C28DD26201F701B7306805206602D2C5
:10011000B101B7306805206602D28701B7306805A3
:10012000206602D28101B7C28230680A2066077455
:1001300008D5E0FDD2B101B7C28630680A20660753
:100140007408D5E0FDD28701B7C28030680A206606
:10015000077408D5E0FDD28101B7C2AFC2AD53E646
:10016000EFC0D0C0E0D2D3D2AFC2CEE52A60072024
:100170007449152A21BB7800790020742EE580305F
:100180007E01F430E50278FF53DACF207E0343DAB4
:1001900020307E0343DA10C2D8C271E580307E0180
:1001A000F430E50279FFC3E89970CB306103752A1A
:1001B00018207403752A18885CD27020740DE52B02
:1001C0006004152B21CB43DA01C2D8207002413ED6
:1001D000A85C206102C270207431C3E894F040032F
:1001E00074F0F8E8C4540F28F87984B70302410B7F
:1001F000C313C3138721200802C313200A06C3C8F0
:1002000098F8410B28F8500374FFF8C3E89565503F
:1002100003E565F88822E52D54066022206B1FE572
:1002200036C333C333F8E564C313C313F9C395224C
:1002300040028922E82522F52250037522FF8522FB
:1002400024A824C3E52495614002A8618825E566B9
:1002500070024182C3E8AA669A5003E8FAE4F9EA18
:10026000C333FBE568F45B29400D2567F8E567605B
:10027000021567400B41820AC3E5679A5002056781
:1002800078FF8826C26FC3E52694F84002D26FC378
:10029000E52594404002D26420CF0AD0E0D0D0437C
:1002A000E610D2AD32C2CF053A7801E52A600530BA
:1002B0007402152AC3E55C94014005755F0041D1C5
:1002C000756000756900E55F2401F55F5003755F97
:1002D000FFD0E0D0D043E610D2AD32C2AF53E67FBC
:1002E0007592FA7593FFC260759104D2AF32C2AFB6
:1002F00053E6EFC2ADC0D0C0E0C0F0D2D3D2AFA8B9
:10030000FBA9FCC2D8307102615553DACF207E03BD
:1003100043DA10307E0343DA20D271E580307E016B
:10032000F420E502612C88278928A18253DACF20A6
:100330007E0343DA20307E0343DA10C2D8C2713024
:100340007402A16E7800E580307E01F430E502A1F0
:100350006E885CA15653DACF207E0343DA20307ECC
:100360000343DA10C271206102812E53DACF207E5E
:100370000343DA10307E0343DA20C2D8D2718857A3
:100380008958C3E89555F8E99556F97B007E087AB7
:1003900000C3E8948CE994005005755B00812088C7
:1003A0002178A2E6A8216055C3E894C8E9940050DA
:1003B00008E4D2E4FB7A0A61FBC3E89468E994019B
:1003C0005008E4D2E3FB7A0F61FBC3E894D0E994D0
:1003D000025008E4D2E2FB7A1E61FBC3E894A0E974
:1003E00094055008E4D2E1FB7A3C61FBC3E89498A1
:1003F000E994085008E4D2E0FB7A787E00C3E895DF
:1004000059FCE9955AFD30E70AECF42401FCEDF4BF
:100410003400FD755B00C3EC9AED9E5003755B01E3
:100420008859895A8557558558567802A156C3E888
:100430009527F8E99528F9307C02A13A307B02A192
:100440003A307A02A1332075028151E9FDE8FC813E
:1004500070E9C313F9E813F8307902A133E9C31343
:10046000F9E813F8307802A133E9C313FDE813FC6F
:0F04700020612CC3EC941CED940240028187EDB7
:10047F00701EC3EC94C850180529E5297002152980
:10048F00C3E529940A5002A16E755C00D270A16E6B
:10049F00E529600215297888E6F97400207F08782D
:1004AF0096B90302789EE624FAFEE43400FFC3EC0B
:1004BF009EFCED9FFD9208B90310A208500720760D
:1004CF0009D27681D9307602C276A2085016B903C6
:1004DF000DECF42401FCEDF43400FD0204F378007C
:1004EF007900A13AB90315EC33FCED33FDC3EC945D
:1004FF000AFCED9400FD50047C007D00C3EC94FFDA
:10050F00ED9400400678FF7900A13AEC8572F0A4D3
:10051F00C5F0A2F733F87900400302055678FF794A
:10052F0000020556E9C313F9E813F8307C0EE960B1
:10053F000278FFC3E81338F8E43400F9C3E894FFF6
:10054F00E99400400278FF885CD270206102A16EAE
:10055F00741FF4552F4BF52FC274EB7002D27475C4
:10056F002A18307403752A0A306102A1822074039D
:10057F0053DAFE207403752B06D0F0D0E0D0D0D222
:10058F00AD43E6103279010205B279030205B27963
:10059F000A0205B2791E0205B279640205B279C862
:1005AF000205B27817E4D5E0FDD8FAD9F6227A140D
:1005BF007B780205D97A107B8C0205D97A0D7BB432
:1005CF000205D97A0B7BC80205D97902E4C286D518
:1005DF00E0FDD287D5E0FDC287D5E0FDD286D5E01C
:1005EF00FDE920E002D2B130E002D281E573D5E01F
:1005FF00FDE920E002C2B130E002C2817496D5E07D
:10060F00FDD9C9EAF8D5E0FDD8FBDBBEC28622C30F
:10061F007C007D0075F00005F0EA33FAEB33FB50F8
:10062F00F6EB13FBEA13FAC3E9FFE8FEE89AF8E9E1
:10063F009BF95004EFF9EEF8B3EC33FCED33FDD535
:10064F00F0DFEDF9ECF822E889F08A20D2D4F8A98E
:10065F00F07B0030F70B7BFFF42401F8E9F4340052
:10066F00F9E88520F0A4ADF0F8E98520F0A4AFF00B
:10067F00FEED2EF974003FFA7C04C3EA13FAE91376
:10068F00F9E813F8DCF48BF030F70AE8F42401F8FA
:10069F00E9F43400F9E889F0C2D4F8A9F02222C3B2
:1006AF00E54113F9E54013F8C3E54498F8E545999A
:1006BF00F9500CC3E89480E994FF40160206E5C395
:1006CF00E8947FE9940050030206E5787F790002F1
:1006DF0006E5788079FF8849894A22E5492546F859
:1006EF00E54A3547F9854A20E4300701F43548FAE1
:1006FF0030E709C3EA94F04015020723C3EA940FC9
:10070F00500302072378FF79FF7A0F02072378003F
:10071F0079007AF0C3E5249561500AC374019524DA
:10072F00500B020741E54A20E70E020741E54A3028
:10073F00E706884689478A482278A5E6FAC3E5493D
:10074F0033F8E54A33F9D156E930E70BC3E8948023
:10075F00E994FF4013E17BC3E8947FE994005002D2
:10076F00E17B787F7900E17B788079FFE820E715DE
:10077F00C3E52398F84009C3E8940140030207A298
:10078F0078010207A2E8F424012523F840030207A9
:10079F00A278FF884B2278A6E6FAA847A948D15637
:1007AF00E930E70CC3E89401E994FF40160207D63D
:1007BF00C3E894FFE9940050030207D678FF79004D
:1007CF000207D6780179FFE920E715C3E54B98F8C2
:1007DF004009C3E8940140030207FD78010207FDB9
:1007EF00E8F42401254BF840030207FD78FF882425
:1007FF002278FFC26420693D206A12D264C3E541AA
:10080F00940A4009C3E52594405002C26479A1E7D8
:10081F006023E541601F74FF8541F0848539F03016
:10082F006A0375F005A4F8C5F0600278FFC3E89578
:10083F00645002A864886322C3E5409440E5419464
:10084F0001E5635003140158046002F563220208A6
:10085F00602275E890227883E6FFE5E820ECF7A8A0
:0F086F00BDA9BE0570C3E57094084052757000B6
:10087E00E9FA79A0E76044EA7007E571601B0208A7
:10088E009BC3E895716010E5715006600C14020868
:10089E00A70460F90208A7E571F571C394A8401B7F
:1008AE007561C0C394054013756180C39405400BF8
:1008BE00756140C39405400375610075BB0622E562
:1008CE0061F460020561E570B4070375BB1E227406
:1008DE003279A787F0A4C5F0A2F733F8C3E8956183
:1008EE004002A8618822882488258826886422757B
:1008FE0040007541F022C2AF75C820A8CCA9CDAA80
:10090E003A30CF010A75C824D2AFAB3BAC3C883B22
:10091E00893CC3E89BF8E99C206908F930670241DD
:10092E0010216DAD3D8A3DF9EA9DFA600478FF799C
:10093E00FFAE3EAF3F8B3E8C3FA83BA93CC3E89E2B
:10094E00F8E99FF9C3E54113FBE54013FAE82AF5F0
:10095E0040E93BF54150067540FF7541FF21B7AAAE
:10096E0040AB41AC40AD417E047F02C3EB940440EA
:10097E00021E1FC3EB940840021E1FC3ED13FDECB5
:10098E0013FCDEF7C3EA9CFAEB9DFBEF6009C3E9AB
:10099E0013F9E813F8DFF7EA28FAEB39FB8A408BF4
:1009AE004150067BFF8B408B41C3EB94025002D229
:1009BE00673069047F0321E27892E6FFC3E537943E
:1009CE008240110FC3E53794A040010FC3EF940688
:1009DE0040027F057E02E541C4540FF9E541C4543F
:1009EE00F0F8E540C4540F28F8C3E89EFAE99400E5
:1009FE00FB4009C3EA9402EB940050047A02E4FB34
:100A0E00415CAA40AB41EBC4FEEAC4540F4EFCC39A
:100A1E00EA9CFAEB9400FBC3E813C313F8EA28FA36
:100A2E00EB3400FB8A408B41C3EB94024002C26759
:100A3E007802EBC4FE7B00EAC4540F4EFAC3EA9868
:100A4E00FA4005C3940250027A027892E6FF3060B3
:100A5E0002415C855192855293D26043E680C3E495
:100A6E009AF8E49BF930670241E8E8FAE9FBD3E92A
:100A7E0013FDE813FC88518952C3EF94036038EFDD
:100A8E0020E00DE82CF8E93DF9ECFAEDFB020AB195
:100A9E00E828F8E939F9C3E82402F8E93400F97ACC
:100AAE00FE7BFFC3EF9403400E8A538B54884D890F
:100ABE004E8C4F8D50611C885389548A4D8B4E8CB1
:100ACE004F8D503069127553F07554FF754FF07598
:100ADE0050FF7551F07552FF611CE8FAD3E813FC14
:100AEE008851C3EF94036020EF20E007E82CF8EC68
:100AFE00FA6108E8282402F87AFEC3EF940340084E
:100B0E008A53884D8C4F611C88538A4D8C4FE568F3
:100B1E00C3335002646BF56830600261267534028F
:100B2E00D26043E680E52D54066034A840A941C347
:100B3E00E913F9E813F8C3E913F9E813F830690477
:100B4E00E92440F9C2AF53E67F759100C3E498F5EE
:100B5E0094E499F595759104D26043E680D2AF2264
:100B6E00D265754300752000306C03752040020B72
:100B7E008DD265754300752040306C03752000786A
:100B8E00017901206720E52D54066002C2657914B3
:100B9E00E541C313700104F8C39414400278143075
:100BAE006904781B791B206010E543600C306903E3
:100BBE00D53404D26D812F712E0543E59B5440B57B
:100BCE002002811930690908C3E89940011861B4FF
:100BDE0020650A08C3E8994002618D61B4C265C2FE
:100BEE00AF53E67F7591003067127594007595FED0
:100BFE00759104D26043E680D2AF618DAE40AF41B5
:100C0E00C3E49EF594E49FF59561FEC3E53394012C
:100C1E005002618D306502618DD802812D61B4C2A2
:100C2E006DC2AF53E67F75910085539485549575CB
:100C3E009104854D92854E93D26043E680D2AFE506
:100C4E002D54066008206A020533020C6B306D0DC0
:100C5E00206C0A206507158115810215192278006E
:0F0C6E003064053065027801E53775F007A4F9A9
:100C7D00E5F028F5F0E9A2F013A2F113A2F213F5B5
:100C8D0037C394785003753778C3E53795384008E6
:100C9D00D266C2B1C287C28130600281A5854F92F2
:100CAD00855093D26043E68022207D16C2AF7542F7
:100CBD0002C286D282306202D281D2AF759F020209
:100CCD000EA5C2AF754202C286D280306202D2B189
:100CDD00D2AF759F02020EA5307243207D20C2AFA8
:100CED00754203900138757B40C281C28030620429
:100CFD00D287A103D286D2AF759F03020EA5C2AFD4
:100D0D00754203900138757B40C2B1C282306204D6
:100D1D00D287A123D286D2AF759F01020EA5207D69
:100D2D0017C2AF754203900113C281306202D287A0
:100D3D00D2AF759F03020EA5C2AF7542039001138A
:100D4D00C2B1306202D287D2AF759F01020EA520CB
:100D5D007D16C2AF754204C282D280306202D28744
:100D6D00D2AF759F01020EA5C2AF754204C280D2EB
:100D7D0082306202D287D2AF759F03020EA5307208
:100D8D0043207D20C2AF754205900127757B04C2BB
:100D9D0087C286306204D2B1A1A9D282D2AF759F2B
:100DAD0002020EA5C2AF754205900149757B01C2C5
:100DBD0087C286306204D281A1C9D280D2AF759F1D
:100DCD0002020EA5207D17C2AF754205900109C222
:100DDD0087306202D2B1D2AF759F02020EA5C2AFAB
:100DED0075420590011DC2873062EBD281D2AF757D
:100DFD009F02020EA5207D16C2AF754206C280D29B
:100E0D0086306202D2B1D2AF759F03020EA5C2AF7A
:100E1D00754206C282D286306202D281D2AF759FF0
:100E2D0001020EA5307243207D20C2AF75420190A4
:100E3D000149757B01C2B1C282306204D281C14FBA
:100E4D00D280D2AF759F01020EA5C2AF754201903F
:100E5D000127757B04C281C280306204D2B1C16F9B
:100E6D00D282D2AF759F03020EA5207D17C2AF753A
:100E7D00420190011DC2B1306202D281D2AF759F85
:100E8D0001020EA5C2AF754201900109C281306207
:100E9D0002D2B1D2AF759F03C26622900107757B56
:100EAD0000C2B1C287C281C282C286C280C2622222
:100EBD00788076FF0876FF0876FF0876FF087603C0
:100ECD000876040876090876030876010876017815
:100EDD008C76010876FF0876FF0876FF0876FF0806
:100EED0076FF0876030876FF0876FF0876FF08760A
:100EFD00250876D00876FA0876FA0876040876FF83
:100F0D0008760108760008767A0876FF08760108DB
:100F1D007601087600087603087600227887E6FFCA
:100F2D00C272BF0302D2727888E6C394036008C20E
:100F3D007DE630E102D27DC27E7889E630E102D2D3
:100F4D007EC3EF94026008758E01D273020F617536
:100F5D008E00C273227880E6149000809378A5F6F7
:100F6D007881E6149000809378A6F67886E6149042
:100F7D00008D9378A7F67886E6F539C39402500371
:100F8D00753902789CE67538FFB402037538A0B444
:100F9D00030375388278A3E61490009A93F566D111
:100FAD00A822227896E6FA7897E6FB7888E6B403CD
:100FBD0005C3EB940EFB307F047A007BFFC3EB9AE5
:100FCD00FCC3948250027C827572000572EC8572AE
:100FDD00F0A4C3E5F0947D40F222D27FF1B012056A
:100FED00A37A007B007C10120599E55C2AFA740047
:100FFD003BFBDCF37C04C3EB13FBEA13FADCF7FEDB
:10100D00C27F120FB022E5EF20E603752000052008
:10101D00903DFFE520146006901FFF1460009304BF
:10102D00600375EF1253D9BF7581C043FF80120560
:10103D009475EF0243B203E5B3240220E70DF521C9
:10104D00E5B120E0068521B343B101120EA87580EC
:10105D003875A4C775F1FF75D4DF7590FF75A500C0
:0F106D0075F20075D50075A0FF75A60075F3002C
:10107C0075D60075B0E475A71B75F4FF75E24112C7
:10108C000EA8E4F8F6D8FD756801120EBD12156AAB
:10109C0078988673753001C2AF1205AD1205BD127A
:1010AC0005A31205C41205A31205CB1205A3121633
:1010BC00831205AD1205AD1205A8C2AF78FA79FA04
:1010CC00308507D9FBD8F7021C00120F29120F62CA
:1010DC00120FAF120FB078988673120EA875881085
:1010EC0075890275C82475910475D84075A8227548
:1010FC00B80275E690759B80759D0075D10E75BC18
:10110C005875BB0675BA1F75E880120594D2AF12DC
:10111C00085D75360053DACF207E0343DA20307E2B
:10112C000343DA1043DA01C2D8C2711205ADD261A1
:10113C007B037A0CE55B70077A0CDB030210C6129A
:10114C0005A32070030210C6C270E55CC394024074
:10115C00E1E52F541F855E5DF55EB55DD5DAD5C230
:10116C006153DACF207E0343DA20307E0343DA105A
:10117C00C2D8C27178A2E67008D274E52F54E0F59B
:10118C002FC2757529001205A8307409C3E529947E
:10119C000A4002D27512059978023074027800C3A5
:1011AC00E55C9840F0C2AF1205BD1205BD1205BD3D
:1011BC00D2AF1205AD754C007888E6B4030241A994
:1011CC00120599788CE6C3940150030212A9E530FC
:1011DC00C3940150030212A9207435C3E55C94FF3B
:1011EC0050030212A9C2AF1205D2D2AF1205A8C386
:1011FC00E55C940150EFC2AF1205BD12059E1205BD
:10120C00BDD2AF1205A8C3E55C94FF40E9021708F4
:10121C007F05D27F120FB01205A8C2AFC27F120F8A
:10122C00B0AE5CC3E55C947FD2AF407B120594C238
:10123C00AF1205D2D2AFDFDA120FE7C3EE94057806
:10124C0097F61205AD1215AC12168B7F0AD27F12CF
:10125C000FB01205A8C2AFC27F120FB0AE5CC3E5CF
:10126C005C947FD2AF50E4120594C2AF1205BD124C
:10127C00059E1205BDD2AFDFD4120FE7EE24037822
:10128C0096F61205AD1215AC1216BA1205A8120F6D
:10129C00B0C3E55C94FF500221E4021708C3E55C7F
:1012AC00954C4003855C4C1205A878017988E7B40D
:1012BC0003027805C3E55C98400221C4C2AF120555
:1012CC00D21205D21205D2D2AF1205AD753000E4A0
:1012DC00F531F5320531E531F4703F0532789AE697
:1012EC007819146012783214600D787D14600878C7
:1012FC00FA146003753200C3E53298401D120EA833
:10130C00120594153275310078998673C2AF1205A7
:10131C00D2D2AF789886731205A812059EE52A7072
:10132C000530740201C678012074027806C3E55CAE
:10133C009840A17888E6C3940360031205A8E52AB7
:10134C0070030210C6C2AF120EA8E4F522F523F505
:10135C0024F525F526F567D2AF7885E6C333F56518
:10136C00E4F544F545F546F547F548F570F52CF5EB
:10137C002DF53775700875BB1E120594120861E5C2
:10138C00E820ECFBA8BDA9BEE97001F88871120831
:10139C006575700875BB1E120F29C2AF7561FF12FF
:1013AC0008DD852261852262852263D2AF75220118
:1013BC00752401752501752601856069756A0178AA
:1013CC0088E6B40307C27D307602D27DD268D2693A
:1013DC00753300120E02120E311208FD120904129E
:1013EC0008FD1209041208FD120B7F1206AD120C37
:1013FC006C120CB6120904120B6E306E031206AE90
:10140C00206703120800306703120847120C6C1295
:10141C000CE5120904120B7F306E031206EA120C53
:10142C006C120D5C120904120B6E306E031207481D
:10143C00120C6C120D8B120904120B7F306E0312FE
:10144C0007A5120C6C120E02120904120861120B81
:10145C006E120C6C120E3112086512090430692FD1
:0E146C00856461856462856069756A0179181E
:10147A007A0CC3E53399400CC269D26A8A35756120
:10148A00FF02149BC3E55C940140030213F40215A6
:10149A0021306A1D206C1AE535147006C26AD26BB7
:1014AA0061F4F535C3E55C940140030213F40215B7
:1014BA0021753600788279A4E760027803C3E55F74
:1014CA00985054307404E52A604D7888E6B40317BE
:1014DA00207D0520760781F130760281F1206C07A4
:1014EA00D26C856461813378F0306C0585646178EB
:1014FA0020C3E54198500261F4306C1BC26CC27D76
:10150A00307602D27DD26A75351285646161F4053E
:10151A0036E55C6002A124753600C2AF120EA878C7
:10152A0087E6FE7602120F297887EEF6E4F522F5B1
:10153A0023F524F525F526F565752C00752D00D2C1
:10154A00AF1205A8120EA878A4E66006D2B1D28717
:10155A00D281307409C3E5369404400201C641DBE6
:10156A00901A0D78201215EEE520B45A0CA3121524
:10157A00EEE520B4A50302158C120EBD1215AC02BD
:10158A0015AB901A0378807B0A1215EEA308DBF9D3
:10159A00901A0F788C7B191215EEA308DBF9901AB2
:1015AA002822C2AF12162D121607901A00740E12B4
:1015BA0015F3A374061215F3A374151215F3901AF2
:1015CA000378807B0A1215F2A308DBF9901A0F78C8
:1015DA008C7B191215F2A308DBF912164012161E9B
:1015EA00901A2822E493F622E6438F01538FFD7561
:1015FA00EF0275B7A575B7F1F0538FFE22438F023C
:10160A00438F0175EF0275B7A575B7F1901A0DF002
:10161A00538FFC22901A0D745AB1F3901A0E74A5C6
:10162A00B1F3227A3079D07820901A40B1EEE520D1
:10163A00F709A3DAF7227A3079D0901A40E7B1F3A2
:10164A0009A3DAF922AB74A875BB01027984BB023B
:10165A00027985BB03027986BB04027992BB050233
:10166A007987BB060279A3BB0702799CBB0802797A
:10167A0088BB09027989E8F7227C051205ADDCFBF3
:10168A0022C2AF1205BD1205C41205CB1205D21231
:10169A00059E1205BD1205C41205CB1205D212050C
:1016AA009E1205BD1205C41205CB1205D2D2AF2275
:1016BA00C2AF1205D21205CB1205C41205BD12051E
:1016CA009E1205D21205CB1205C41205BD12059E43
:1016DA001205D21205CB1205C41205BDD2AF22AE35
:1016EA0074AF75C2AF1205BD1205BD1205BD120554
:1016FA009EDEF21205D212059EDFF8D2AF22D18BFE
:10170A00D183D183757401757501757600D1E97C31
:10171A0005AD5C1205ADC3ED955C70F5C3E55C944F
:10172A0001400AC3E55C94FF4032021744D14FB12D
:10173A00ACD18BC2AF75EF12D183DCD50576C3E588
:10174A00769403500280C6D1830575E5741490001F
:10175A009F93F808C3E57598500280AED183D18370
:10176A000574C3E574940A5002809C120EBDB1AC94
:07177A00C2AF75EF12D1832D
:0319FD00021013C2
:101A00000E0615FFFFFFFF0304090301015AA5019C
:101A1000FFFFFFFFFF03FFFFFF25D0FAFA04FF01DE
:091A2000007AFF0101000300FF40
:101A4000235475726E696779343041232020202039
:101A500023424C48454C4923463331302320202033
:101A60002020202020202020202020202020202076
:101C0000C2AFC2D353D9BF7581C043B20343FF8073
:101C1000752438752503B1C975EF0275E24043F1AB
:101C20002053A4DF75D4FFD2857DFA780379E67C52
:101C300010752200752300901DD67B0675249875BB
:101C400025013085028142208508D8FBD9F9DCF7CF
:101C500081B4308508D8FBD9F9DCF781B4B189E4C7
:101C600093A3C39A6004DDC381B4DBDBB17B600264
:101C7000812B7B08E493FAA3B15CDBF87A30B15C8A
:101C8000752200752300B17BEAFCEBFDC3ED94FEE9
:101C9000400EB17B8A278B28ED30E0048A828B834B
:101CA000B17B7AC270D8C3ED94FE601350CEBD00F4
:101CB00025EC60097520007521FF0200008100A855
:101CC00027A9280809D804D90281D3B17FEA89AAB3
:101CD000F281C50D81A0C3ED94035049EDA2E092BD
:101CE000007AC5C3E5829400E583941C50902000DF
:101CF00010438F02438F0175B7A575B7F1F030001F
:101D00001FA827A9280809438F01538FFDD804D99C
:101D100002A12089AAE275B7A575B7F1F0A3A10DBC
:101D2000538FFC817C7AC1BD030CE493A3FAB140CC
:101D3000DCF8B138817C817EAA22AB23B15CEBFA5E
:101D4000EA6222752608C3E52313F523E52213F57D
:101D50002250066323A0632201D526EAB1C9B1C986
:101D600075260AEAF4200102D285300102C285B14B
:101D7000C9C3134002C201D526EB22B17FEAFB2082
:101D80008502A17F308502A184752608AE24AF2587
:101D9000C3EF13FFEE13FEB1CDB1C9C3EA13308513
:101DA000024480FA30E703632201C3E52313F523DD
:101DB000E52213F52250066323A0632201D526D91C
:101DC000E52265236523F52222AE24AF250E0FDE22
:101DD000FEDFFCD20122424C48656C693437316326
:041DE000F3100601F5
:00000001FF
